:060000000A128A11122809
:10000800FE00030EF1000408F2000A08F300831250
:1000180003137F08F4000A128A11D82A0A128A11D7
:100028000F2E8B010730831603139F00283083128D
:10003800031385008316031385010130831203130C
:100048008600013083160313860083120313870189
:10005800831603138701043081007D308312031354
:10006800AC002C08FC00FB01B301B401AF01B001E6
:10007800B201B101FA01063081008B160B168B17FD
:10008800051406160A128A1167250A128A118312A4
:100098000313A30100300A128A11DD250A128A11FE
:1000A80056300A128A11B8250A128A1183120313CC
:1000B800A301A30A00300A128A11DD250A128A1147
:1000C80023300A128A11B8250A128A1183120313DF
:1000D800AE0114302E02031C7228732875288B2851
:1000E8008B288230AD00DD30AC00AC0B7928AD0B2D
:1000F80079287E28013083120313AC002C08AE0740
:1001080014302E02031C89288A2875288B28A301FD
:1001180000300A128A11DD250A128A1123300A12C8
:100128008A11B8250A128A1183120313A301A30A9C
:1001380000300A128A11DD250A128A1101300A12CA
:100148008A11B8250A128A1183120313AE010A30E4
:100158002E02031CB028B128B328C928C928823028
:10016800AD00DD30AC00AC0BB728AD0BB728BC2810
:10017800013083120313AC002C08AE070A302E029C
:10018800031CC728C828B328C928A30100300A12AD
:100198008A11DD250A128A1101300A128A11B8253E
:1001A8000A128A1183120313A301A30A00300A1248
:1001B8008A11DD250A128A1134300A128A11B825EB
:1001C8000A128A1183120313AE010A302E02031C8D
:1001D800EE28EF28F128072907298230AD00DD3005
:1001E800AC00AC0BF528AD0BF528FA2801308312CA
:1001F8000313AC002C08AE070A302E02031C052995
:100208000629F1280729A30100300A128A11DD25E1
:100218000A128A1134300A128A11B8250A128A1170
:1002280083120313A301A30A00300A128A11DD25E1
:100238000A128A1145300A128A11B8250A128A113F
:1002480083120313AE010A302E02031C2C292D2918
:100258002F29452945298230AD00DD30AC00AC0B93
:100268003329AD0B33293829013083120313AC002D
:100278002C08AE070A302E02031C432944292F29D3
:100288004529A30100300A128A11DD250A128A11B4
:1002980045300A128A11B8250A128A1183120313EB
:1002A800A301A30A00300A128A11DD250A128A1155
:1002B80012300A128A11B8250A128A1183120313FE
:1002C800AE010A302E02031C6A296B296D29832985
:1002D80083298230AD00DD30AC00AC0B7129AD0B49
:1002E80071297629013083120313AC002C08AE075C
:1002F8000A302E02031C812982296D2983290030A6
:100308000A128A11CB210A128A110A128A111B2693
:100318000A128A118F29831203133208031D9529A3
:10032800AF290430AC002C08FA000A128A111B26E7
:100338000A128A1101300A128A11CB210A128A1173
:10034800831203133308AC002C08B400B301AF01C7
:10035800B001B201AF293108031DB3298F290A1250
:100368008A1126260A128A1102300A128A11CB2112
:100378000A128A1183120313B401B301AF01B00149
:10038800B1018F298F298F290A128A111228831205
:100398000313AB00A30100300A128A11DD250A12EB
:1003A8008A117C300A128A11B8250A128A1183121E
:1003B8000313AB08031DE129E229E92983300A1256
:1003C8008A11B8250A128A11E929831203132B0806
:1003D800013A031DF029F129F9293308303E0A12A0
:1003E8008A1131260A128A11F929831203132B085C
:1003F800023A031D002A012A072A86300A128A11A6
:10040800B8250A128A110E300A128A11B8250A1262
:100418008A1176300A128A11B8250A128A118312B3
:100428000313AB08031D192A1A2A212A82300A123B
:100438008A11B8250A128A11212A831203132B085C
:10044800013A031D282A292A5E2A0A30A000003012
:10045800A1002F08A900AA012908A2002A08A300C0
:100468000A128A118D240A128A1183120313200892
:10047800303E0A128A1131260A128A110A30831272
:100488000313A0000030A1002F08A900AA01290821
:10049800A2002A08A3000A128A1101250A128A1149
:1004A800831203132008303E0A128A1131260A12D9
:1004B8008A115E2A831203132B08023A031D652A48
:1004C800662A6D2A85300A128A11B8250A128A11FD
:1004D8006D2A83120313A301A30A00300A128A119A
:1004E800DD250A128A1167300A128A11B8250A1204
:1004F8008A1183120313AB08031D832A842A8B2ACB
:1005080082300A128A11B8250A128A118B2A83129C
:1005180003132B08013A031D922A932AC82A0A308A
:10052800A0000030A1003008A900AA012908A200F3
:100538002A08A3000A128A118D240A128A1183122A
:1005480003132008303E0A128A1131260A128A1132
:100558000A3083120313A0000030A1003008A9005C
:10056800AA012908A2002A08A3000A128A11012553
:100578000A128A11831203132008303E0A128A11C4
:1005880031260A128A11C82A831203132B08023A49
:10059800031DCF2AD02AD72A85300A128A11B825F6
:1005A8000A128A11D72A08000B1DDB2ADC2A022B23
:1005B8000B11063081000130FC02FC08031DE52AFE
:1005C800E62AEE2A7D30F0007008FC000430F000C6
:1005D8007008FB007B08031DF22AF62A0130FB0293
:1005E8008514F82A8510F82A7A08031DFC2A002B9E
:1005F8000130FA020515022B0511022B8B1C052B65
:10060800062BBA2B8B10F9010E2B0130F000700865
:10061800F9070E2B061C112B122B092B132B463016
:100628007902031C182B192BBA2B5B30790203189B
:100638001E2B1F2BBA2BB301AF01B001F701F80134
:10064800F6010D307602031C2A2B2B2B2D2B8A2B1F
:100658008A2B003006180130F0007008F50032309F
:10066800F0007008F900382B06183B2B3C2B4E2B5A
:100678007508031D402B4E2B0130F7070318F80AA5
:100688000030F80701300310F70DF80DFF3E031D89
:10069800472B692B061C512B522B5F2BF508031D8A
:1006A800562B572B5F2B01300310F70DF80DFF3E2B
:1006B800031D582B692B0130F902031D642B652B90
:1006C800382B692B692B382B382BF908031D6D2B18
:1006D8006E2B702B8A2B8A2B7830F0007008F9006B
:1006E800782B0130F902782B0230790203187D2B20
:1006F8007E2B752B7F2B0130F0007008F6070D302C
:100708007602031C882B892B2D2B8A2B7908031D35
:100718008E2BB52B01300310F80CF70CFF3E031D90
:100728008F2B77083F39F0007008B00006300310AF
:10073800F80CF70CFF3E031D9B2B77081F39F000C0
:100748007008AF0005300310F80CF70CFF3E031DCE
:10075800A72B77080139F0007008B300B201B20A7C
:10076800BA2BB101B10ABA2BBA2BBA2B7408FF0005
:1007780073088A0072088400710E8300FE0E7E0ED4
:02078800090066
:1008000004308A000408840A82070034203420342B
:1008100020342034203420344C3455344B3441348B
:100820002034203420342034203420340034203448
:100830002034203431343934373434342D343234A4
:1008400030343134333420342034203420340034F4
:1008500020347334743461346E34643461347234EB
:1008600064347534203452344334353420342034E5
:10087000003420342034283443342934203465347F
:100880004B3461346D3453346F34663474342034F3
:1008900020340034203462347934203452346134CA
:1008A000663461346C34203453347A3475346C34A7
:1008B0006334203400342034543465347334743455
:1008C000653472342034703469346C346F34743469
:1008D0006F347734203400342034203420342034F2
:1008E0002034203420342034203443344F344D34E9
:1008F0003A34203400344134443452343A342034CD
:1009000000345334593453343A34203400342D34C1
:100910002D34003458345834003483120313A601A4
:10092000A11F932C942C9C2CA009A109A00A0319A7
:10093000A10AA601A60A9C2CA31F9F2CA02CAA2CBE
:10094000A209A309A20A0319A30A0130A4002408DA
:10095000A606AA2CA701A801210820040319B12C7E
:10096000B22CEF2CA501A50AC12C01300310A00D5B
:10097000A10DFF3E031DB62C0130A4002408A507DD
:10098000C12CA11FC42CC52CB52CC72CC72C0130E1
:100990000310A70DA80DFF3E031DC82C210823023C
:1009A000031DD42C20082202031CD72CD82CE02CA9
:1009B0002008A2022108031CA303A3022714E02C91
:1009C00001300310A10CA00CFF3E031DE12C0130EF
:1009D000A502031DEC2CED2CC72CEF2CEF2C2608C8
:1009E000031DF32CF92CA709A809A70A0319A80AC3
:1009F000F92C2808A101A1072708A001A007002DB4
:100A0000080083120313A601A31F072D082D102D24
:100A1000A209A309A20A0319A30AA601A60A102D76
:100A2000A11F132D142D1A2DA009A109A00A031925
:100A3000A10A1A2D2108200403191F2D202D552D40
:100A4000A501A50A2F2D01300310A00DA10DFF3E19
:100A5000031D242D0130A4002408A5072F2DA11F5C
:100A6000322D332D232D352D352D21082302031D45
:100A70003B2D20082202031C3E2D3F2D462D200831
:100A8000A2022108031CA303A302462D0130031078
:100A9000A10CA00CFF3E031D472D0130A502031D34
:100AA000522D532D352D552D552D2608031D592D0D
:100AB0005F2DA209A309A20A0319A30A5F2D230827
:100AC000A101A1072208A001A007662D080041305E
:100AD00083120313A600EE30A500A50B6D2DA60B07
:100AE0006D2D00008312031386108611061130301D
:100AF0008700861586110D30A600FB30A500A50BDA
:100B00007F2DA60B7F2D842D303083120313870099
:100B1000861586114230A500A50B8C2D00003030C3
:100B2000831203138700861586114230A500A50B9A
:100B3000972D000038300A128A113C260A128A11B9
:100B400008300A128A113C260A128A110A128A11E6
:100B5000F1250A128A1106300A128A113C260A125D
:100B60008A110C300A128A113C260A128A110800D6
:100B700083120313A400CF2D240884000A128A11C3
:100B800000240A128A110A128A1131260A128A11C5
:100B9000013083120313A3002308A407CF2D2408D8
:100BA00084000A128A1100240A128A110038031DD7
:100BB000DA2DDB2DBC2DDC2D080083120313A500DC
:100BC0002308A40006300310A40DFF3E031DE32DEF
:100BD00025082407803E0A128A113C260A128A112F
:100BE000080001300A128A113C260A128A110730C5
:100BF00083120313A4007D30A300A30BFD2DA40BCF
:100C0000FD2D080083120313A1002108870086151B
:100C100086114230A000A00B0B2E00000800FA0144
:100C2000FB01AF01B001B101B201B301B401830115
:100C30000A128A1115288312031385112130A0008E
:100C4000A00B202E831203138515080083120313B3
:100C500085122130A000A00B2B2E831203138516C2
:100C6000080083120313A200861422080A128A11B4
:100C700002260A128A11080083120313A2008610AA
:0E0C800022080A128A1102260A128A1108009E
:02400E0071FF40
:00000001FF
